:100000000C94460018950000189500001895000003
:10001000189500001895000018950000189500002C
:10002000189500001895000018950000189500001C
:10003000189500001895000018950000189500000C
:1000400018950000189500001895000018950000FC
:1000500018950000189500001895000018950000EC
:1000600018950000189500001895000018950000DC
:1000700018950000189500001895000018950000CC
:100080001895000018950000189500008FEF8DBF9F
:10009000C0EEE8ED4E2E80E18EBFD0E1F0E15F2EA4
:1000A000EEEFFFE0A0E0B1E0A89584B7082E877FCF
:1000B00084BF88E1992781BD91BD88278D933197B1
:1000C000E9F785E089B980E08093900088E18AB9FA
:1000D00066248CEF84BB0E949C0CBE9A81E28FBD8B
:1000E00081E08EBD86E886B980E087B9BC98BD9A6C
:1000F000179A129813981498159889980E94F70CDB
:100100001A9A1C9A1D9A1B9AC49A919A80E080931D
:1001100006018EE496E0A1E0B1E08D939C931F98D8
:1001200082E08093030181E080930401882780931B
:100130000501E2E6FCE10E94890D0E946E0CE1E0FF
:10014000F0E00E94750CA6E0B1E08C9199279093A5
:100150004900809348001F9A82E08093030181E068
:1001600080930401882780930501ECE6FCE10E945E
:10017000890D0E946E0C8FEF90E090934900809360
:100180004800E1E0F0E00E94750CBD9AE6E7FCE172
:100190000E94890D0E94580C0E945F0CA8E0B1E0FB
:1001A000E4E9FCE10E94890D0E94690DA8E0B1E03C
:1001B0000E94170EA9E4B1E08C9381E080933A018C
:1001C0004091490100913A01041718F011F00C9484
:1001D0001E0280913A01E8E0F1E001E00A93A6E313
:1001E000B1E00E94FC0DA6E3B1E08C91A8E3B1E080
:1001F0008C930E94F70C00913801003211F00C949E
:100200001E0184E08093030181E08093040188272C
:1002100080930501EEEBFCE10E94890D0E946E0CBB
:10022000E4ECFCE10E94890D0E94580C0E945F0CD6
:100230008EE591E00E948D0C0C941602009138011D
:100240000C3311F40C9416020091380143E2041BA4
:10025000A9E3B1E00C9381E08093030181E08093F6
:10026000040180E080930501A6E3B1E00E94680CE0
:10027000E4ECFCE10E94890D0E946E0CA0ECB0E160
:10028000E8E3F1E00E94AF0D0E94660CE4ECFCE1B3
:100290000E94890D0E946E0CA0ECB0E1E9E3F1E050
:1002A0000E94AF0D0E94660CA6E3B1E00E94520CC2
:1002B000E4ECFCE10E94890D0E94580CA0ECB0E136
:1002C000E8E3F1E00E94AF0D0E94500CE4ECFCE189
:1002D0000E94890D0E94580CA0ECB0E1E9E3F1E026
:1002E0000E94AF0D0E94500C0E945F0CECE4F4E001
:1002F0000E94890DA9E3B1E08C9199270E94790DA4
:10030000ACE3B1E00E94690D83E08093030181E0DA
:1003100080930401882780930501ACE3B1E00E943B
:10032000680CACE3B1E00E94170EAAE4B1E08C9334
:1003300081E080934B0140914A0100914B010417E9
:1003400018F011F00C94EF0180914B01ECE3F1E017
:1003500001E00A93ACE4B1E00E94FC0DACE4B1E032
:10036000E6ECFCE10E94890D0E941D0E11F00C9438
:10037000CB01BD9AE4E1F5E082E390E00197C59AF4
:100380000E94800CC5980E94800C482F492BB1F721
:10039000C59A0C94DB01BD9AE4E1F5E086E990E0B2
:1003A0000197C59A0E94800CC5980E94800C482F26
:1003B000492BB1F7C59A40914A0100914B010417AE
:1003C00010F00C94E70182E390E00E948D0CABE406
:1003D000B1E08C918F5F8C9310F40C949B01009191
:1003E0003A0141E0040FABE3B1E00C9380913B0193
:1003F000E8E0F1E001E00A93A6E3B1E00E94FC0D21
:10040000A6E3B1E08C91A8E3B1E08C9300913801B0
:100410000C3311F40C94120286E990E00E948D0CCA
:100420000C94160282E390E00E948D0CAAE3B1E0E6
:100430008C918F5F8C9310F40C94E00084EF91E02A
:100440000E948D0C0C94CE00F894FFCF2E2E2E2EF1
:100450002E2E2E2E2E002E2E2E2E2E2E2E2E2E0018
:100460002E2E2E2E2E2E2E2E2E002E2E2E2E2E2EDA
:100470002E2E2E002E2D2D2D2D2E002D2E2D2D2EFF
:10048000002D2E2D2D2E2D002E2E2E2E2E2E2E2EEC
:100490002E002E2E2E2E2E2E2E2E2E002D2D2E2EDA
:1004A0002D2D002D2E2E2E2E5F002E2D2E2D2E2D9D
:1004B000002D2E2E2D2E002D2D2D2D2D002E2D2DEF
:1004C0002D2D002E2E2D2D2D002E2E2E2D2D002EDD
:1004D0002E2E2E2D002E2E2E2E2E002D2E2E2E2E9A
:1004E000002D2D2E2E2E002D2D2D2E2E002D2D2DBE
:1004F0002D2E002D2D2D2E2E2E002E2E2E2E2E2E7C
:100500002E2E2E002E2E2E2E2E2E2E2E2E002E2E67
:100510002E2E2E2E2E2E2E002E2E2E2E2E2E2E2E29
:100520002E002E2E2D2D2E2E002E2E2E2E2E2E2E49
:100530002E2E002E2D002D2E2E2E002D2E2D2E0097
:100540002D2E2E002E002E2E2D2E002D2D2E002E87
:100550002E2E2E002E2E002E2D2D2D002D2E2D0078
:100560002E2D2E2E002D2D002D2E002D2D2D002E6A
:100570002D2D2E002D2D2E2D002E2D2E002E2E2E2B
:10058000002D002E2E2D002E2E2E2D002E2D2D0076
:100590002D2E2E2D002D2E2D2D002D2D2E2E00003A
:1005A0000108080000000000000000000000065FD5
:1005B00006000000000703000703000000247E245B
:1005C0007E24000000242B6A120000000063130840
:1005D0006463000000364956205000000000070305
:1005E0000000000000003E41000000000000413E0D
:1005F0000000000000083E1C3E0800000008083E05
:10060000080800000000E060000000000008080882
:1006100008080000000060600000000000201008D2
:1006200004020000003E5149453E00000000427FA8
:10063000400000000062514949460000002249493B
:1006400049360000001814127F100000002F49499D
:1006500049310000003C4A4949300000000171095D
:1006600005030000003649494936000000064949A3
:10067000291E000000006C6C000000000000EC6C03
:10068000000000000008142241000000002424247F
:100690002424000000004122140800000002015937
:1006A00009060000003E415D551E0000007E11114C
:1006B000117E0000007F494949360000003E41415B
:1006C00041220000007F4141413E0000007F494936
:1006D00049410000007F090909010000003E41492D
:1006E000497A0000007F0808087F00000000417F71
:1006F0004100000000304040403F0000007F0814EF
:1007000022410000007F404040400000007F020482
:10071000027F0000007F0204087F0000003E41418C
:10072000413E0000007F090909060000003E4151DA
:10073000215E0000007F0909196600000026494972
:10074000493200000001017F01010000003F4040EC
:10075000403F0000001F2040201F0000003F403CA1
:10076000403F000000631408146300000007087095
:1007700008070000007149454300000000007F4168
:100780004100000000020408102000000000414168
:100790007F000000000402010204000080808080CD
:1007A0008080808000000307000000000020545477
:1007B00054780000007F444444380000003844442A
:1007C0004428000000384444447F0000003854545A
:1007D0005408000000087E09090000000018A4A4C5
:1007E000A47C0000007F0404780000000000007D6D
:1007F00040000000004080847D000000007F102841
:10080000440000000000007F40000000007C04184D
:1008100004780000007C04047800000000384444A0
:100820004438000000FC444444380000003844448C
:1008300044FC0000004478440408000000085454BC
:100840005420000000043E4424000000003C4020EE
:100850007C000000001C2040201C0000003C603098
:10086000603C0000006C10106C000000009CA06058
:100870003C000000006454544C00000000083E415D
:10088000410000000000007700000000000041412E
:100890003E0800000002010201000000003C262387
:1008A000263C0000001EA1E121120000003D402076
:1008B0007D000000003854545509000000205555B3
:1008C00055780000002055545578000000205555FB
:1008D000547800000020575557780000001CA2E211
:1008E00022140000003855555508000000385554B2
:1008F0005508000000385555540800000000017CE0
:100900004100000000000279420000000000017C6C
:1009100040000000007029242970000000782F2575
:100920002F780000007C5454554500000034547C5E
:1009300054580000007E097F4949000000384545B1
:1009400039000000003845443900000000394544B2
:1009500038000000003C41217D000000003D4120A6
:100960007C000000009CA1603D000000003D424270
:100970003D000000003C41403D000000001824669E
:100980002400000000483E494962000000292A7CFA
:100990002A290000007F0916781000000040887E98
:1009A0000902000000205455557800000000007D29
:1009B000410000000038444539000000003C40215F
:1009C0007D000000007A090A71000000007A1122FF
:1009D0007900000000085555555E0000004E515149
:1009E0004E0000000030484D40200000003C040450
:1009F0000404000004040404041C00000017084C54
:100A00006A500000001708342A7800000000307D8A
:100A10003000000000081400081400000014080052
:100A2000140800004411441144110000AA55AA55AD
:100A3000AA550000BBEEBBEEBBEE0000000000FFBD
:100A400000000000080808FF000000000A0A0AFF72
:100A50000000000008FF00FF0000000008F808F890
:100A6000000000000A0A0AFE000000000AFB00FF66
:100A70000000000000FF00FF000000000AFA02FE74
:100A8000000000000A0B080F00000000080F080F0C
:100A9000000000000A0A0A0F00000000080808F819
:100AA000000000000000000F080800000808080F00
:100AB00008080000080808F808080000000000FF07
:100AC000080800000808080808080000080808FFCF
:100AD00008080000000000FF0A0A000000FF00FFF5
:100AE00008080000000F080B0A0A000000FE02FAC6
:100AF0000A0A00000A0B080B0A0A00000AFA02FAA6
:100B00000A0A000000FF00FB0A0A00000A0A0A0A9B
:100B10000A0A00000AFB00FB0A0A00000A0A0A0B84
:100B20000A0A0000080F080F080800000A0A0AFA5B
:100B30000A0A000008F808F808080000000F080F6B
:100B4000080800000000000F0A0A0000000000FE74
:100B50000A0A000000F808F80808000008FF00FF73
:100B6000080800000A0A0AFB0A0A00000808080F21
:100B700000000000000000F808080000FFFFFFFF71
:100B8000FFFF0000F0F0F0F0F0F00000FFFFFF00CA
:100B900000000000000000FFFFFF00000F0F0F0F1C
:100BA0000F0F0000001824241824000000FE4A4AF9
:100BB00034000000007F01010300000000027E02FB
:100BC0007E020000006355496300000000182424E1
:100BD0001C04000000FC20201C0000000008047819
:100BE000040000000008557755080000003E494900
:100BF0003E000000004C7202724C00000022555969
:100C00003000000000182418241800000018247E6A
:100C100024180000001C2A2A2A000000003C0202BE
:100C20003C000000002A2A2A2A0000000000242E8E
:100C30002400000000514A4A4400000000444A4A8F
:100C400051000000000000FC020400000020403FB2
:100C5000000000000008082A0808000000241224F0
:100C60001200000000060909060000000000181824
:100C70000000000000000800000000000030403EBE
:100C80000202000000010E010E00000000090D0A22
:100C900000000000003C3C3C3C0000000210200032
:100CA0000000000000000000000000000000000044
:100CB0000000000000000000000000000000000034
:100CC0000000000000007CFFFF7C0000000000002E
:100CD00000000000000000333300000000000000AE
:100CE00000000000003C3C00003C3C000000000014
:100CF00000000000000000000000000000000000F4
:100D000000001090F07E1E90F07E1E10000000008B
:100D100000021E1F03021E1F03020000000000004D
:100D20000000000078FCCCFFFFCCCC880000000065
:100D300000000000040C0C3F3F0C0F0700000000F7
:100D40000000001C1C1C80C0E070381C0E0000005D
:100D50000000181C0E070301001C1C1C00000000F2
:100D60000000000000B8FCC6E23E1C0000000000CD
:100D7000000000001F3F3121371E1C3622000000FA
:100D8000000000000000273F1F00000000000000DE
:100D90000000000000000000000000000000000053
:100DA000000000F0FCFE0701010000000000000050
:100DB000000000030F1F382020000000000000008A
:100DC0000000000000010107FEFCF0000000000030
:100DD00000000000002020381F0F0300000000006A
:100DE000000000004C5CF0FCFCF05C4C00000000DB
:100DF00000000000060701070701070600000000C9
:100E000000000000808080F0F08080800000000002
:100E1000000000000101010F0F01010100000000AE
:100E200000000000000000000000000000000000C2
:100E300000000000000000B8F8780000000000008A
:100E400000000000808080808080808000000000A2
:100E5000000000000101010101010101000000008A
:100E60000000000000000000000000000000000082
:100E700000000000000000383838000000000000CA
:100E80000000000000000080C0E070381C0E06006A
:100E9000000000181C0E0703010000000000000005
:100EA000000000F8FE060383C363331EFEF8000053
:100EB000000000071F1E3331303030181F070000BC
:100EC00000000000000C0C0EFFFF000000000000FE
:100ED00000000000003030303F3F30303000000074
:100EE0000000001C1E07030383C3E3773E1C0000C1
:100EF00000000030383C3E373331303030300000B5
:100F00000000000C0E07C3C3C3C3C3E77E3C000050
:100F10000000000C1C383030303030391F0E00001B
:100F2000000000C0E070381C0E07FFFF000000004A
:100F3000000000030303030303033F3F0303000018
:100F40000000003F7F636363636363E3C383000068
:100F50000000000C1C383030303030381F0F0000DB
:100F600000000000C0F0F8DCCEC7C3C3C38000009F
:100F7000000000070F1F393030303030391F0F00AC
:100F8000000000030303030303C3F33F0F03000048
:100F9000000000000000303C0F03000000000000D3
:100FA000000000BCFEE7C3C3C3E7FEBC00000000B6
:100FB00000000F1F393030303030391F0F00000073
:100FC0000000003C7EE7C3C3C3C3C3E7FEFC0000D0
:100FD0000000000000303030381C0E070300000015
:100FE00000000000000000707070000000000000B1
:100FF000000000000000001C1C1C0000000000009D
:101000000000000000000070707000000000000090
:10101000000000000000009CFC7C000000000000BC
:101020000000C0E0F0381C0E0703000000000000C4
:101030000000000103070E1C383000000000000013
:101040000000000060606060606060606000000040
:10105000000000000606060606060606060000005A
:1010600000000000000003070E1C38F0E0C0000084
:1010700000000000000030381C0E070301000000D3
:101080000000001C1E070383C3E3773E1C00000022
:1010900000000000000000373700000000000000E2
:1010A0000000F8FE07F3FB1BFBFB07FEF800000047
:1010B00000000F1F183337363737360301000000A2
:1010C0000000000000E0FC1F1FFCE000000000002A
:1010D000000000383F0706060606073F38000000FC
:1010E000000000FFFFC3C3C3C3E7FEBC0000000055
:1010F0000000003F3F3030303030391F0F0000001B
:10110000000000F0FC0E07030303070E0C000000B4
:10111000000000030F1C38303030381C0C00000079
:10112000000000FFFF03030303070EFCF0000000B4
:101130000000003F3F30303030381C0F030000000B
:1011400000000000FFFFC3C3C3C3C3C30303000009
:10115000000000003F3F3030303030303030000091
:10116000000000FFFFC3C3C3C3C3C30303000000E9
:101170000000003F3F0000000000000000000000F1
:1011800000000000F0FC0E0703C3C3C3C7C6000085
:1011900000000000030F1C38303030303F3F0000AB
:1011A000000000FFFFC0C0C0C0C0C0FFFF000000C3
:1011B0000000003F3F0000000000003F3F00000033
:1011C00000000000000303FFFF0303000000000015
:1011D000000000000030303F3F30300000000000D1
:1011E0000000000000000000000000FFFF00000001
:1011F0000000000E1E3830303030381F070000006D
:10120000000000FFFFC0E0F0381C0E0703000000E4
:101210000000003F3F000103070E1C3830000000B3
:10122000000000FFFF0000000000000000000000C0
:101230000000003F3F3030303030303030000000B0
:10124000000000FFFF1E78E0E0781EFFFF000000B6
:101250000000003F3F0000010100003F3F00000090
:10126000000000FFFF0E38F0C00000FFFF0000008C
:101270000000003F3F00000003071C3F3F0000004C
:10128000000000F0FC0E070303070EFCF000000056
:10129000000000030F1C383030381C0F0300000022
:1012A000000000FFFF8383838383C7FE7C00000070
:1012B0000000003F3F0101010101010000000000AA
:1012C000000000F0FC0E070303070EFCF000000016
:1012D000000000030F1C3830363E1C3F3300000076
:1012E000000000FFFF8383838383C7FE7C00000030
:1012F0000000003F3F010103070F1D3830000000D0
:101300000000003C7EE7C3C3C3C3C78E0C000000CF
:101310000000000C1C3830303030391F0F00000046
:1013200000000000030303FFFF03030300000000AD
:10133000000000000000003F3F000000000000002F
:10134000000000FFFF000000000000FFFF000000A1
:10135000000000071F3830303030381F0700000011
:10136000000000073FF8C00000C0F83F0700000081
:101370000000000000010F3E3E0F010000000000D1
:10138000000000FFFF000080800000FFFF00000061
:101390000000003F3F1C060303061C3F3F00000007
:1013A000000000030F1C30E0E0301C0F03000000C1
:1013B000000000303C0E030101030E3C3000000031
:1013C000000000030F3CF0C0C0F03C0F0300000021
:1013D000000000000000003F3F000000000000008F
:1013E00000000003030303C3E3331F0F03000000E7
:1013F000000000303C3E33313030303030000000EF
:101400000000000000FFFF030303030000000000D2
:1014100000000000003F3F3030303000000000008E
:10142000000E1C3870E0C0800000000000000000CA
:101430000000000000000103070E1C18000000005F
:1014400000000003030303FFFF0000000000000092
:10145000000000303030303F3F000000000000004E
:10146000006070381C0E070E1C3870600000000011
:10147000000000000000000000000000000000006C
:10148000000000000000000000000000000000005C
:10149000000000C0C0C0C0C0C0C0C0C0C0C000000C
:1014A0000000000000003E7E4E0000000000000032
:1014B000000000000000000000000000000000002C
:1014C0000000000040606060606060E0C0000000FC
:1014D0000000001C3E3333333333333F3F00000002
:1014E000000000FFFFC060606060E0C0800000009E
:1014F0000000003F3F3030303030381F0F00000018
:1015000000000080C0E06060606060C0800000009B
:101510000000000F1F383030303030180800000055
:1015200000000080C0E0606060E0C0FFFF000000DD
:101530000000000F1F3830303030303F3F000000D7
:1015400000000080C0E06060606060C0800000005B
:101550000000000F1F3B333333333313010000000F
:10156000000000C0C0FCFEC7C3C3030000000000B1
:1015700000000000003F3F000000000000000000ED
:1015800000000080C0E06060606060E0E00000009B
:1015900000000003C7CECCCCCCCCE67F3F000000DF
:1015A000000000FFFFC0606060E0C080000000003D
:1015B0000000003F3F00000000003F3F000000002F
:1015C00000000000000060ECEC00000000000000E3
:1015D000000000000030303F3F30300000000000CD
:1015E000000000000000000060ECEC0000000000C3
:1015F000000000000060E0C0C0FF7F0000000000AD
:101600000000000000FFFF0080C0E060000000005C
:1016100000000000003F3F03070F1C3830000000AF
:1016200000000000000003FFFF00000000000000B9
:10163000000000000030303F3F303000000000006C
:10164000000000E0C0E0E0C0C0E0E0C080000000BA
:101650000000003F3F00003F3F00003F3F00000010
:1016600000000000E0E060606060E0C0800000001A
:10167000000000003F3F00000000003F3F0000006E
:1016800000000080C0E060606060E0C0800000009A
:101690000000000F1F3830303030381F0F000000BE
:1016A000000000E0E06060606060E0C0800000007A
:1016B000000000FFFF0C181818181C0F070000008E
:1016C00000000080C0E06060606060E0E00000005A
:1016D000000000070F1C181818180CFFFF0000006E
:1016E00000000000E0E0C060606060E0C00000005A
:1016F000000000003F3F000000000000000000006C
:1017000000000000C0E06060606060400000000019
:10171000000000001133333333333F1E000000005C
:10172000000000006060FEFE6060600000000000DD
:101730000000000000001F3F30303030000000008B
:10174000000000E0E0000000000000E0E000000019
:101750000000000F1F3830303030183F3F000000CD
:1017600000000060E0800000000080E060000000F9
:101770000000000001071E38381E070100000000AD
:10178000000000E0E00000E0E00000E0E000000019
:10179000000000071F381C0F0F1C381F0700000037
:1017A0000000000060E0C0800080C0E06000000039
:1017B0000000000030381D0F070F1D3830000000FA
:1017C000000000000060E080000080E06000000099
:1017D00000000000000081E77E1E070100000000FD
:1017E000000000006060606060E0E06020000000D9
:1017F0000000000030383C3633313030300000001B
:10180000000080C0FC7E070303030000000000000E
:10181000000000011F3F70606060000000000000D9
:101820000000000000FFFF000000000000000000BA
:1018300000000000003F3F0000000000000000002A
:101840000000000000030303077EFCC080000000CE
:101850000000000000606060703F1F010000000099
:1018600000000010180C040C1810180C04000000E4
:101870000000000000000000000000000000000068
:1018800000000080C0603018183060C08000000088
:101890000000000707060606060606070700000008
:1018A000A0ECB0E18D91882311F00CD0FBCF08950E
:1018B0000E946F0D802D11F005D0FACF08958DE0B4
:1018C00001D08AE05D9BFECF8CB90895A0ECB0E119
:1018D0008D91882311F00FD0FBCF08950E946F0DDA
:1018E000802D11F008D0FACF089588EE93E015D03E
:1018F0003197D9F708950C940B0D3197F1F70895AE
:10190000AE2FBF2F11974A2F4B2BE1F70895689404
:1019100062F80895E89462F80895EF93FF93EE2734
:10192000E82BE92B31F0EDECFAE03197F1F7019774
:10193000D1F7FF91EF910895442718D0AD98AC9A54
:10194000AA9884E699270E948D0C9FEF9ABBAD9AC6
:101950002ED014FCFDCF02D04FEF08D08FE30FD074
:1019600080EC0DD080E40BD088EB09C0403420F02F
:10197000AF9AAE9840540895AE9AAF980895AB9838
:1019800001C0AB9AEF93FF93EAE0F0E00E947D0C78
:10199000FF91EF918BBBAC98AA9AEF93FF93E2E093
:1019A000F0E00E947D0CFF91EF91AA980895AB980A
:1019B00004D017FCFCCF0895AB9A99279ABB9FEFF0
:1019C0009BBBEF93FF93EAE0F0E00E947D0CFF9158
:1019D000EF91AC9AAA9AEF93FF93E2E0F0E00E94B5
:1019E0007D0CFF91EF9119B2AA989ABB08954427F4
:1019F000BDDF02D04FEFBADF00E080E4C0DF88EB4C
:101A0000800FBDDF10E48827BCDF1A95E1F703954E
:101A1000083099F70895EF93FF931BB61F925091EA
:101A200003015F9370900401E0910101F0910201C4
:101A30000024EE0FFF1F001C0BBE0E946F0D202D17
:101A40000E946F0D302D0E946F0D002D0E946F0DB2
:101A50008052482F0E940B0EE40FF51F27D0709282
:101A60000401732F409104015091030129D00E9479
:101A70006F0D802D50910501552309F0809581DF70
:101A8000509104015395509304017A9559F7509160
:101A900003015395509303012A9509F75F915093E1
:101AA00003011F901BBEFF91EF91089518F42BB610
:101AB00023942BBE089518F42BB62A942BBE0895B8
:101AC0004A955A9553DF88EB850F59DF80E4840FE0
:101AD00056CF0E946F0D0D920020D9F70895D8952A
:101AE000319628F48F938BB783958BBF8F9100200D
:101AF0000895882311F4992329F00E946F0DE9F7C6
:101B00000197D9F708950F9301E00BBF0F918894C7
:101B100008950F930027F9CF0F9302E0F6CF0F93AC
:101B200003E0F3CF000F111F221F331F089500950C
:101B30001095209530950F5F1F4F2F4F3F4F089501
:101B4000019110810EC001911191219130810BC042
:101B50000191108117FF05C03FEF2FEF04C00081F6
:101B600011272227332737FF03C0E1DF8DE28D9352
:101B7000CF93DF93CF92DF92EF92AA24BB24CC24A1
:101B8000DD24EE2440E2CAE0DD2755E093E38881BE
:101B9000890F87FD9F7083FD907F891B89935A95DC
:101BA000A9F7C0DFAA1CBB1CCC1CDD1CEE1C4A958F
:101BB00051F7E894EFE0FF2782910ED0EB30E0F789
:101BC0001EF068948A2D0CD088278D93EF90DF90BB
:101BD000CF90DF91CF910895982F829501D0892FD2
:101BE0008F70805D26F0803309F4089568948D939A
:101BF000089588278D93089509919191992351F023
:101C00008A95D9F7319781918D930A9519F0882398
:101C1000D1F70895EECFFF935527F8E0469508F4E5
:101C2000500F57954795FA95D1F7FF9108958FEF8B
:101C300083959D919923E1F70895689401C0E894F4
:101C4000AF93BF938D9116F0919103C00E946F0DD9
:101C5000902D891718F011F48823A1F7BF91AF9147
:101C60000895484F4C4420505752000052454C4173
:101C700053452021000053656E6463686172202023
:101C800043686172636F6465202044617461696EAA
:101C9000646578004142434445464748494A4B4CB5
:101CA0004D4E4F505152535455565758595A203152
:101CB000323334353637383930203F3E3C0073708C
:081CC0006163650020002E00A5
:00000001FF
